:0E0000000C9498000C9400000C9400000C94DA
:10000E0000000C9400000C9400000C9400000C9462
:10001E0000000C94F3000C9400000C9400000C945F
:10002E0000000C9400000C9400000C9400000C9442
:10003E0000000C9400000C9400000C9400000C9432
:10004E0000000C94000020202020202020202020C2
:10005E00202020202020000080C01027E80364000C
:10006E000A0001000010000110000100312D333490
:10007E003536373839303132333435360000322D9B
:10008E003334353637383930313233343536000083
:10009E00332D333435363738393031323334353613
:1000AE000000202020204C434420546573742020EF
:1000BE002020002020202020202020202020202052
:1000CE0020202000202020202048616C6C6F2020F2
:1000DE00202020200020202020312E205A65696CFF
:1000EE0065202020200020202020322E205A6569F5
:1000FE006C652020202000313233343536373839C4
:10010E006162636465666700120060017A00120026
:10011E0072018C00120084019E000200960166009E
:10012E000000F894EE27ECBBF1E0FBBFEBBFE5BFA0
:10013E00F8E1F1BDE1BD8DE0A2E0BB27ED938A951C
:10014E00E9F780E094E0A0E6ED930197E9F7E6E1A8
:10015E00F1E085919591009761F0A591B59105908B
:10016E001590BF01F00105900D920197E1F7FB018B
:10017E00F0CFEFE5EDBFE4E0EEBFC0E6D1E00C94CA
:10018E00F4000A9300E000E0033018F5E981E15035
:10019E00E017A8F00E94E903E02FA0E6B1E0F0E03E
:1001AE00BF93AF93A2E1B0E00E946104AF91BF9103
:1001BE00EA0FFB1FFA93EA930E940E0208C00E94F8
:1001CE00E903E4E5F0E0FA93EA930E9418020F5F68
:1001DE00DBCF0881229608951895E0E0EBBBEABBD1
:1001EE00E8BBE7BBE5BBE4BBE2BBE1BBE3BFE2BF01
:1001FE00ECBFEFBDE5E0EEBDE0E0EDBDECBDE7BD73
:10020E00E6BDEBBDEABDE9BDE8BDE2BDE5BDE4BDC1
:10021E00E3BDE5BFE4BFE4E0E9BFE0E8E8B9E0E054
:10022E00E0BFE0E1EA930E9434027894E0E6F1E068
:10023E00FA93EA93E0EBF0E0FA93EA9380E00E94FF
:10024E00BE032496E2E7F1E0FA93EA93E1ECF0E0E4
:10025E00FA93EA9380E00E94EE03E0EBF0E0FA936B
:10026E00EA9380E00E94BE032496E2E7F1E0FA935F
:10027E00EA93E2EDF0E0FA93EA9380E00E94EE0357
:10028E00E3EEF0E0FA93EA9380E00E94BE03249638
:10029E00E2E7F1E0FA93EA93E4EFF0E0FA93EA93FF
:1002AE0080E00E94EE03E5E0F1E0FA93EA9380E04D
:1002BE000E94BE032496E2E7F1E0FA93EA93E2EDA0
:1002CE00F0E0FA93EA9380E00E94EE03E0EBF0E0B8
:1002DE00FA93EA9380E00E94BE032496E2E7F1E0EF
:1002EE00FA93EA93E5E0F1E0FA93EA9380E00E9454
:1002FE00BE032496E2E0EA930E94C800E4EFF1E028
:10030E00FA93EA930E944D0491CFFFCFFFE0FA9546
:10031E00F1F70895AAB3AF70AABBD99AD8980E94E4
:10032E008D01DA9A0E948D01A9B3DA980E948D018F
:10033E00DA9A0E948D01DA98A7FDF1CF0895A07F79
:10034E00AB2BABBBDA9A0E948D01DA980E948D011D
:10035E000895D998AAB3A76FAABBBBB3BF70A881E3
:10036E000E94A601A881A2950E94A601D99A219663
:10037E000895DA9A0E948D01E9B3DA980E948D01F0
:10038E00E07F08950E948D010E94C001AE2F0E9451
:10039E00C001D998E295EA2B08950E949101E88157
:1003AE00F0E0EA56FE4FE081A981EA0FEA930E943F
:1003BE00B00149805880229608950E949101E2E092
:1003CE000E94FF03ECE00E94FF03E1E0EA930E942B
:1003DE00B001E0E05E2E4E2E0895EF93FF93A881BC
:1003EE006894AA3021F0E8944394641438F453943A
:1003FE00E0E0EA935A920E94D4012EF08BDFD89A55
:10040E00A881AA93A6DFFF91EF9121960895F98115
:10041E00E881A191AA2319F0AA93DFDFFACF2296E1
:10042E000895E881F981C895002021F031960A924D
:10043E00D4DFF9CF22960895AA27BB271197F1F79B
:10044E000895D998AAB3A76FAABBBBB3BF70A881F2
:10045E000E94A601D99A21960895DA98D8986880B4
:10046E00E881E058E0939801E881E054E093990127
:10047E000E9404040E9404040E942302E0E80E94E9
:10048E000A040E940A040E940A04EA930E942802A7
:10049E000E9404040E942302E8E20E941104E4E098
:1004AE000E941104E5E80E941104AAB3AF70AABB22
:1004BE00D99A0E94C901E53011F0E0E009C00E940E
:1004CE009101E6E0EA930E94B0010E94E401E1E0AE
:1004DE00219608955F9BFECFACB108955D9BFECF34
:1004EE00A881ACB921960895A881B9810E946904AA
:1004FE00309749F00E9469043196ED93FC93319741
:10050E00AA81A08304C0EA81EA930E947502239611
:10051E00089526970E94710400E0E889F9893196C2
:10052E00E88BF98B3197E4913E2FE03011F40C9467
:10053E00BA03E02FE03039F4353211F401E002C095
:10054E000E9416040FC1E130B1F4353221F40E943D
:10055E00160400E007C102E050E010E03D3211F455
:10056E0011E000C13B3211F45BE2FCC0303211F4F9
:10057E0050E2F8C002C0E23039F440E003E030331C
:10058E0011F41068EFC004C0E33011F00C94B903FD
:10059E00303310F03A3308F009C0A42FEAE0EA9F96
:1005AE00E02D4E2FE32FE0534E0FDCC0E32FE3364A
:1005BE0031F40E941D04EC910E942404D2C0E33752
:1005CE0041F40E941D040E942B040E9438040E2F39
:1005DE000AC0E03761F40E941D040E942B040E94A1
:1005EE0042040E2F186012601F7720E038C0E436E8
:1005FE0011F0E93611F4146002C0E53731F4E8E683
:10060E00F0E0EE83FF8305E00DC0E83511F41860CD
:10061E0004C0E83711F00C94B803E2E7F0E0EE8383
:10062E00FF8304E012FF15C00E941D040E9469049E
:10063E00EA87FB87AA85BB8510972CF40E945D0480
:10064E00EA87FB875DE2503011F00F5F01C01B7F20
:10065E0006C00E941D040E946904EA87FB8710FDF4
:10066E0011C0041778F417FF08C012FF04C01B7FD7
:10067E00352F015001C030E301C030E20E94160454
:10068E004150EFCF202F11FF1AC02030B9F013FFC9
:10069E0008C0EE81FF813196EE83FF833197E4919E
:1006AE0005C0AE81BF81ED91AE83BF83EA930E94F8
:1006BE003204403009F041502150E7CF4AC030E3B8
:1006CE00EE81FF813296EE83FF8332970E946D0496
:1006DE00E887F987AA85BB85AE17BF0720F03F5F75
:1006EE00AE1BBF0BC9F7AA87BB87E9E3E31728F454
:1006FE0013FF02C0395F01C0395D14FD1DC0E0E378
:10070E00E31730F0A885B985A130E0E0BE0711F4FB
:10071E0010610AC0421710F010FF01C011C030E284
:10072E0017FF0AC030E3106112FF06C01B7F5A93F9
:10073E0092D0403009F0415072D0403009F0415013
:10074E002150A885B985E1E0F0E0EA17FB0708F42F
:10075E00B6CF10FF06C0403021F04150E0E26DD020
:10076E00FACF00E0DACE0E94780462960895FF92E6
:10077E00F82E22971A930A93DE010E9459040A2F2B
:10078E001B2FDE0116960E9459040E946904EA830B
:10079E00FB83DE0114960E9459040E946904FA93A9
:1007AE00EA931A930A93FE013696FA93EA930E94FD
:1007BE009002AA81BB81E0E0EC9319810881249616
:1007CE00FF900895E0E0EA930A930C94D401CFDFF2
:1007DE002496E2E0EA930E94C800E4EFF1E0FA9377
:1007EE00EA930E944D04E0E6F1E0FA93EA9308954D
:1007FE00EA930E94B0010C9491010E942302E0E260
:10080E00EA930C942802EA930E9428020E94230283
:10081E00E0E30895EA930E94B0010C9423023A9308
:10082E00ED85FE85FA93EA930C947B02AE85BF8527
:10083E001497AE87BF8714960895EA93ED85FE85CB
:10084E00FA93EA930C947B020E946904EE83FF8371
:10085E00FA93EA930895ED85FE85FA93EA930C9444
:10086E007B02A991B991EE27FF276D91662311F0B6
:10087E003196FBCF0895AA27BB27E991F9910590F0
:10088E00002011F01196FBCFFD010895E991F99129
:10089E00309639F080ED97E00197F1F7A8953197F2
:1008AE00C9F708950024AF0DB01D0895E095F09599
:1008BE0031960895FA9FF02DEB9FF00DEA9FE02DF3
:1008CE00F10D0895ED91FC91119708950590F49115
:1008DE00E02D08955A934A933A932A931A930A93C2
:1008EE0008955D814C813B812A811981088108958B
:00000001FF
